S01200006F7064726163687420432E737265635A
S113000045C000004BC0000049C0000047C00000CC
S113001045C0000043C0000041C000003FC00000D4
S11300203DC000003BC0000039C0000037C00000E4
S113003035C0000033C0000031C000002FC00000F4
S11300402DC000002BC0000029C0000027C0000004
S113005025C0000023C0000021C000001FC0000014
S11300601DC000001BC0000019C0000017C0000024
S113007015C0000013C0000011C000000FC0000034
S11300800DC000000BC0000009C0000011241FBEF9
S1130090CFEFD0E1DEBFCDBF67D088C0B1CF20E0C5
S11300A030E008C0E3ECF9E03197F1F700C000005C
S11300B02F5F3F4F28173907ACF308958FEF87BBA5
S11300C087B3877F87BB88B3816088BB82E58DB99E
S11300D008958FB9779BFECF089598B321E030E05F
S11300E002C0220F331F8A95E2F72095292328BBEB
S11300F0089598B321E030E002C0220F331F8A959F
S1130100E2F7292B28BB0895CF93DF93D82FC62F6E
S113011080E0E3DF8D2FDDDF8C2FDBDF80E0E9DFA4
S1130120DF91CF91089580E0D8DF89E0D2DF8FEFAF
S1130130D0DF80E0DEDF80E0D0DF8AE0CADF84E069
S1130140C8DF80E0D6DF80E0C8DF8BE0C2DF87E075
S1130150C0DF80E0CEDF80E0C0DF8CE0BADF81E08A
S1130160B8DF80E0C6CF0895CF9381E087BBA6DFD8
S1130170DADFC1E004C060E08C2FC6DFCF5FC93096
S1130180D0F388EE93E08BDFC1E007C06C2F8C2F97
S1130190BBDF88EE93E083DFCF5FC930B8F388EE2E
S11301A093E07DDF81E090E0CF910895F894FFCF54
S9030000FC
